:020000040800F2
:1000000020090020D500000851200008391F0008F1
:1000100000000000000000000000000000000000E0
:100020000000000000000000000000004B2E00084F
:100030000000000000000000492E00089D2E00086E
:10004000000000000000000000000000E7000008C1
:10005000E7000008E7000008E7000008E7000008E4
:100060000000000000000000000000000000000090
:10007000E7000008E7000008E700000800000000B3
:1000800000000000E700000800000000E700000892
:10009000000000000000000000000000E700000871
:1000A00000000000E700000800000000E700000872
:1000B0000000000000000000000000000000000040
:1000C0000348854600F028F9004800479D300008A5
:1000D000200900200448804704480047FEE7FEE767
:1000E000FEE7FEE7FEE7FEE7A52E0008C1000008D8
:1000F000D2B201E00270401C491EFBD270470022C0
:10010000F6E710B513460A4604461946FFF7F0FF16
:10011000204610BDF8B502464A40D40F42004B00BD
:1001200052085B089A4202D20246084611464A002B
:1001300023D0C30D4A00DDB2120EAD1A202D35DAE0
:1001400049020126490AF6058A19002C00D05242BC
:1001500020214F1B1146B9402A411018C20D9A4266
:1001600021D0002C17D0012D08DCDA05801AD20F1F
:100170008019D207DBB200F095F8F8BDDA05801AD5
:10018000012340001B06C01880185A428018CA0F6D
:100190001043490007E04908C2071143DA05801AF5
:1001A00080194008801800F075F8F8BD6100012240
:1001B000511A001BF7E70122D2075140AAE701229A
:1001C000D2075040A6E7024670B54A40D30FDB077E
:1001D00040002DD04A002AD0010E140E0002120257
:1001E0000919400A520A8418E50104465443000ADA
:1001F000120A2E045043A4194219200CC543AA1810
:10020000120C0125AD03521C521912047F3924042B
:1002100000D0521C104301D44000491EC2B20C064B
:10022000C0092018401C4008802A02D003E00020AA
:1002300070BD40084000002900DA0020184370BD5E
:10024000C217C10F504010B54018CA0796230021AD
:1002500000F028F810BD70B50446002903D0002036
:100260002022012310E0002801D00020C043C04616
:10027000C0460DE02546D5408D4205D30D4695403C
:10028000641B1D46954040191546521E002DF1DC99
:10029000214670BD002904DA401C490001D1400804
:1002A0004000704770B40024050C05D110240004F0
:1002B00002D1002921D01124050E01D100020834F9
:1002C000050F01D10001241D850F01D18000A41C60
:1002D000002801DB4000641C002908D020252E1BCB
:1002E0000D46F540A14000D00121294308430106F5
:1002F0001B1B000ADB1D02D5002070BC7047DB050C
:10030000181880180029F8DA401C4900F5D170BC93
:100310004008400070470000064C0125064E05E0ED
:10032000E36807CC2B430C3C98471034B442F7D316
:10033000FFF7CAFE90310008B0310008FFE7FEE782
:1003400080B590B007A801902421FFF7D8FE01984E
:100350000021029106910591049103910F220792C9
:10036000012212020B920C910F4A12880D920891F1
:100370000E91099101F02AFA002803D0FFE7FFF758
:10038000DDFFFFE70720039000210491059106910E
:1003900003A801F069F8002803D0FFE7FFF7CEFFBC
:1003A000FFE710B080BDC0460001FF1F80B58CB0D4
:1003B0000A9009910892079303A9002008700998F0
:1003C00000F09BF8002804D0FFE70BA9012008707B
:1003D0008FE00899087849780902401806A9019128
:1003E00008800A9802F02EF801980088000400287E
:1003F00008D5FFE70698404206A9088003A9012016
:100400000870FFE70898017905A8017006A90A8815
:10041000130904AA1370497849074B0E049919432C
:100420001170007800901F280CD0FFE700983F283B
:1004300015D0FFE700985F281ED0FFE700987F28BF
:1004400027D034E006980007C00FFFF7F9FE0290AE
:1004500002983F210906FFF7B6FE02902EE00698AB
:100460000007800FFFF7ECFE029002987D21C9057E
:10047000FFF7A9FE029021E006980007400FFFF762
:10048000DFFE029002981F214906FFF79CFE0290B2
:1004900014E006A800880F210840FFF7D1FE029063
:1004A00002987B21C905FFF78EFE029006E00799AE
:1004B000002008600BA9012008701AE0002104A8A0
:1004C0004056FFF7BDFE0299FFF724FE029003A8F5
:1004D0000078002806D0FFE702990020FFF76BFEA6
:1004E0000290FFE70298079908600BA900200870A6
:1004F000FFE70BA800780CB080BD82B00090009898
:100500000078282804D1FFE701A90020087003E043
:1005100001A901200870FFE701A8007802B0704728
:1005200080B586B00490049800782838414248414C
:1005300003A9009108700498072101F0CDFD02463F
:10054000009802A90A700978049AD279891A4A4255
:10055000514101AA11700078002809D0FFE701A8D5
:100560000078002804D0FFE705A90020087003E008
:1005700005A901200870FFE705A8007806B080BD36
:1005800080B586B00490039102920298002803D1AE
:10059000FFE71C480290FFE7049801F053FF04981E
:1005A000039901F045FE0498BE2102F0B3F8002043
:1005B0000190FFE7019808280BDCFFE7049801F0A1
:1005C00012FF0299019A8854FFE70198401C01909C
:1005D000F0E70298082101F07FFD014668460170AE
:1005E00000780299097A884204D0FFE705A9012022
:1005F000087003E005A900200870FFE705A800784F
:1006000006B080BD1005002080B584B00290019135
:1006100001990020C872FFE70198F02101F042FF24
:10062000012801D0FFE70BE001980299C27AD200BD
:10063000891801F0B5FD0199C87A401CC872EBE732
:100640000198C07A012804DBFFE703A900200870A5
:1006500003E003A902200870FFE703A8007804B0B4
:1006600080BD80B58AB00890079106A802700798EF
:10067000FFF743FF002804D0FFE709A90120087015
:100680004DE0089801F0DEFE0898079901F0D0FDD2
:100690000898BE2102F03EF8089801F0A4FE0898E0
:1006A00001F0A1FE089801F09EFE05A900910870D6
:1006B000089801F098FE04A901910870089801F0CB
:1006C00092FE03A90291087006980870089801F03C
:1006D000B9FE0898079901F0ABFD08984E2102F089
:1006E00019F800990898097802F014F80199089807
:1006F000097802F00FF802990898097802F00AF8D0
:10070000089801F09FFE0898079901F091FD08985C
:10071000482101F0FFFF09A900200870FFE709A8A0
:1007200000780AB080BD80B582B00190019801F0D8
:1007300089FE0198CC2101F0EDFF0198442101F0E0
:10074000E9FF002002B080BD80B584B0029000F0C7
:10075000FDFD0190FFE7029801F014FE00280DD185
:10076000FFE700F0F3FD0199401A0849884204D3DD
:10077000FFE703A90320087004E0ECE703A90020C9
:100780000870FFE703A8007804B080BDEF02000006
:10079000B0B590B0009204460098149A0E940D9152
:1007A0000CA908800BA803800AAB1A700C9A04AB42
:1007B0001A70497803AA11700B9902AA1170407837
:1007C00001A908700D98FFF798FE002804D0FFE7F4
:1007D0000FA90120087087E00E9801F033FE0E98F3
:1007E0000D9901F025FD0E98BE2101F093FF0E98A2
:1007F00001F0F9FD0E9801F0F6FD0E9801F0F3FD01
:1008000009A908700E9801F0EEFD08A908700E986D
:1008100001F0E9FD07A908700E9801F0E4FD0E98BB
:1008200001F0E1FD06A908700E9801F0DCFD05A9B4
:1008300008700AA80078C007002804D0FFE70498D1
:1008400009A90870FFE70AA800788007002804D5E6
:10085000FFE7039808A90870FFE70AA80078400797
:10086000002804D5FFE7029806A90870FFE70AA848
:1008700000780007002804D5FFE7019805A9087053
:10088000FFE70E9801F0DEFD0E980D9901F0D0FC07
:100890000E984E2101F03EFF0E9809A9097801F04B
:1008A00039FF0E9808A9097801F034FF0E9807A9BE
:1008B000097801F02FFF0E9806A9097801F02AFFA8
:1008C0000E9805A9097801F025FF0E9801F0BAFDF0
:1008D0000E980D9901F0ACFC0E98482101F01AFF1A
:1008E0000FA900200870FFE70FA8007810B0B0BD76
:1008F00080B584B0029001910298002804D1FFE7EE
:1009000003A90120087014E00198002804D1FFE732
:1009100003A9012008700CE0029801994860019930
:100920000A6B0298904769460870009803A90870FE
:10093000FFE703A8007804B080BD80B584B00290C2
:10094000029800788007C00F002804D1FFE703A9B0
:100950000120087034E0029A5068114608311032C4
:10096000FFF70EFE014601A80170007800280ED1A5
:10097000FFE702990878012210430870029908786D
:10098000FB221040087003A90020087018E00298AC
:100990000078C00700280AD0FFE70299886B401C46
:1009A000886302990878042210430870FFE70299CF
:1009B0000878FE221040087003A902200870FFE7A3
:1009C00003A8007804B080BD80B584B0029002987E
:1009D000002804D1FFE703A90120087034E0029841
:1009E00000788007C00F002804D1FFE703A9012089
:1009F000087029E00298FFF7A0FF014601A80170E6
:100A00000078002804D0FFE7019803A908701BE0D4
:100A1000029B5868194608311A4610321C33FFF7FA
:100A2000C5FC014601A801700078002808D0FFE746
:100A30000299C86B401CC863019803A9087003E0C1
:100A400003A900200870FFE703A8007804B080BD68
:100A500080B584B002900298002804D1FFE703A972
:100A60000120087029E00298FFF767FF01A90870CC
:100A7000029800784007C00F00281AD0FFE7B3485B
:100A80001049FFF7C1FD002804D0FFE703A90120AA
:100A9000087012E002990A6B48689047002804D059
:100AA000FFE703A90120087007E003A900200870F0
:100AB00003E003A902200870FFE703A8007804B050
:100AC00080BDC046BC00002010B58AB008900898D0
:100AD000002804D1FFE709A90120087016E0089951
:100AE000203102A801901CC91CC01CC91CC0089858
:100AF0004821FFF704FB0199089820301CC91CC04D
:100B00001CC91CC009A900200870FFE709A80078CB
:100B10000AB010BD80B586B004900391029203988C
:100B2000002804D1FFE705A9012008704BE00498D4
:100B3000002804D1FFE705A90120087043E00498CC
:100B40000399486003990020C8608860029908688A
:100B50004A680399CA608860039A50681146083150
:100B60001032FFF70DFD014601A801700078002842
:100B700020D1FFE704980299039A2D23D25CFFF756
:100B800070FD014601A801700078002809D1FFE737
:100B90000399087802221043087005A90020087004
:100BA00011E003990878FD2210400870019805A90A
:100BB000087008E003990878FD2210400870019839
:100BC00005A90870FFE705A8007806B080BD000001
:100BD00080B584B0029001910298002804D1FFE70B
:100BE00003A90120087016E00198002804D1FFE74E
:100BF00003A9012008700EE0029801992C228A5C5A
:100C0000D300A94AD218FFF785FF694608700098FB
:100C100003A90870FFE703A8007804B080BDC046B0
:100C200080B58CB00A9009910A98002804D1FFE79A
:100C30000BA90120087085E00998002804D1FFE77E
:100C40000BA9012008707DE000200790069009980C
:100C50002721415C06A80190017009992622895C30
:100C6000417009992522895C817009992422895C47
:100C7000C17009992322895C017109992222895C3A
:100C8000417109992122895C817109992022895C2D
:100C9000C171FFF745FC002804D0FFE70BA9012034
:100CA00008704FE005A90820087000200490039008
:100CB000FFE703980A99C97A88422CDAFFE705A969
:100CC0000820087000200290FFE70298072815DC32
:100CD000FFE70398C10074484018029A805C06A997
:100CE000895C884205D1FFE70598401E05A9087078
:100CF000FFE7FFE70298401C0290E6E705A80078AE
:100D0000002803D1FFE70398049004E0FFE703986D
:100D1000401C0390CDE705A8007800280ED1FFE71E
:100D20000A980999049AD3005F4AD218FFF7F2FE95
:100D300008A9087008980BA9087003E00BA9012006
:100D40000870FFE70BA800780CB080BD18000020E9
:100D500080B58EB00C900B910C98002804D1FFE761
:100D60000DA9012008709AE00B98002804D1FFE734
:100D70000DA90120087092E00B98008D09A9087058
:100D80000B982921405C08A908700B98408D07A991
:100D900008700B982B21405C06A9087005A900205B
:100DA000087004A908700090FFE700980C99C97AB0
:100DB000884268DAFFE70C980099CA003A49891816
:100DC00001AAFFF7DDFB01460AA8017000780028A0
:100DD00004D0FFE70A980DA9087060E00B98008D19
:100DE000002813D0FFE701A8807809A90978884274
:100DF0000BD1FFE701A8C07808A90978884204D17F
:100E0000FFE705A901200870FFE703E005A901201D
:100E10000870FFE70B98408D002813D0FFE701A86A
:100E2000807907A9097888420BD1FFE701A8C0792A
:100E300006A90978884204D1FFE704A901200870B7
:100E4000FFE703E004A901200870FFE705A8007888
:100E5000002813D0FFE704A8007800280ED0FFE791
:100E60000C980B99009AD3000F4AD218FFF752FE44
:100E70000AA908700A980DA9087010E0FFE7009809
:100E8000401C009091E70B990020C86088600B9986
:100E90000876486108610DA901200870FFE70DA8D8
:100EA00000780EB080BDC0461800002080B588B024
:100EB000069005A8017004A802700698002804D1C5
:100EC000FFE707A9012008704AE00698FFF72BFC0E
:100ED000014603A801700078002804D0FFE70398BA
:100EE00007A908703CE005A80078012809D1FFE7B0
:100EF0000698FFF729FC03A90870039807A9087052
:100F00002EE005A80078022826D1FFE700200190F6
:100F100004A8007800901F280CD0FFE700983F2815
:100F20000BD0FFE700985F280AD0FFE700987F28E2
:100F30000AD00CE05E2001900AE0BC20019007E09E
:100F4000FF207830019003E00748019000E0FFE7C0
:100F5000019800F077F8FFE7039807A90870FFE70A
:100F600007A8007808B080BDEE02000010B588B078
:100F7000069005A8018004A8028003A803700698C3
:100F800000788007C00F002804D1FFE707A90120DF
:100F900008703FE00698FFF7D0FC014602A80170F8
:100FA0000078002804D0FFE7029807A9087031E014
:100FB000069948680831002405AA125F04AB1B5F3C
:100FC00003AC24780094FFF7E3FB014602A801700C
:100FD0000078002808D0FFE70699486C401C486458
:100FE000029807A9087015E0069A50681146083162
:100FF0001032FFF7C5FA014602A8017000780028F8
:1010000004D0FFE7029807A9087003E0029807A937
:101010000870FFE707A8007808B010BD82B0019003
:101020000199074848430090FFE700BFFFE7009899
:10103000411E00910028F8D1FFE702B07047C0467A
:10104000B80B000080B584B0039000F07FF90290E7
:10105000039801900198401C002806D0FFE7EB4858
:101060000168019840180190FFE7FFE700F06EF972
:101070000299401A0199884201D2FFE7F6E704B0CD
:1010800080BDC04688B00790069100200590FFE71C
:10109000069800680599C840002800D132E10698FA
:1010A0000068059A012191400840049004980028A6
:1010B00000D123E106984068022805D0FFE7069892
:1010C0004068122820D1FFE707980599C9088900D0
:1010D0004018006A039005984007C00E0F21814018
:1010E0000398884303900698016905984007C00E4D
:1010F000814003980843039003980799059AD20802
:10110000920089180862FFE7079800680390059825
:101110004100032002468A400399914303910699B6
:1011200049680140059840008140039808430390B6
:101130000398079908600698406801280FD0FFE7D8
:101140000698406802280AD0FFE7069840681128F0
:1011500005D0FFE70698406812282CD1FFE70798D2
:1011600080680390059840000321814003988843DC
:1011700003900698C1680598400081400398084391
:101180000390039807998860079840680390059832
:1011900001218140039888430390069840681021FC
:1011A000084001090598814003980843039003987B
:1011B00007994860FFE70798C068039005984000CA
:1011C000032181400398884303900698816805981D
:1011D0004000814003980843039003980799C86032
:1011E0000698C079C006002800D486E0059803213F
:1011F000884345494058039005988007C00E0F2149
:101200008140039888430390079805210907884285
:1012100003D1FFE7002002900CE007993B4A012030
:10122000022300939142019001D00098019001980F
:101230000290FFE7029905988007C00E814003984D
:101240000843039003980599032291432E4A88503E
:101250002F480068039004990398884303900698E8
:101260008079C007002805D0FFE704990398084358
:101270000390FFE70398264908602648006803901A
:101280000499039888430390069880798007002882
:1012900005D5FFE70499039808430390FFE70398F7
:1012A0001C4908601C48006803900499039888430F
:1012B000039006988079C006002805D5FFE70499B9
:1012C000039808430390FFE7039813490860134805
:1012D00000680390049903988843039006988079E6
:1012E0008006002805D5FFE704990398084303907A
:1012F000FFE7039809490860FFE7FFE70598401CEE
:101300000590C5E608B07047601802400004005020
:10131000801802408418024000180240041802405D
:1013200083B0029001A8018068460270007800280E
:1013300005D0FFE701A800880299886104E001A8B0
:10134000008802998862FFE703B07047054800688B
:101350007047C0462D480268024908688018086036
:101360007047C0461805002080B582B001A9002052
:101370000870032000F00EF8002804D0FFE701A950
:101380000120087002E000F043F8FFE701A80078B0
:1013900002B080BD80B584B0039002A9002008701F
:1013A0001A480068002829D0FFE7BD48006801906E
:1013B000164801687D20C000FEF74DFF01460198E8
:1013C000FEF749FF00F048FC002812D1FFE7039820
:1013D000032809D8FFE703990022D04300F036F82C
:1013E0000398AB49086003E002A901200870FFE7F9
:1013F00003E002A901200870FFE703E002A9012031
:101400000870FFE702A8007804B080BD0C0000203F
:1014100082B0FFE70B48026801210A4302600068BE
:10142000084001900198FFE7FFE7074802680121A3
:1014300009070A4302600068084000900098FFE72F
:1014400002B07047401002403C10024080B584B0AA
:10145000034603A8037002910192002140560299AD
:1014600000F0F8FD04B080BD80B584B00290019119
:101470000298002804D1FFE703A901200870FBE0CF
:1014800001987F49096801221140884221D9FFE76C
:101490007B49086801229043019A10430860FFF7D6
:1014A00055FF0090FFE77648006801210840019948
:1014B00088420DD0FFE7FFF749FF0099401A7549B0
:1014C000884204D3FFE703A903200870D4E0EAE7C9
:1014D000FFE7029800788007002817D5FFE70298F9
:1014E00000784007002807D5FFE7B04908680722C1
:1014F000120310430860FFE7AC4908680F2212028C
:101500009043029A926810430860FFE702980078BF
:10151000C007002861D0FFE70298406801280BD17E
:10152000FFE7A94800684003002804D4FFE703A9A7
:1015300001200870A0E02CE00298406800280BD140
:10154000FFE7A14800684005002804D4FFE703A98D
:101550000120087090E01BE00298406804280BD13D
:10156000FFE7494800688007002804D4FFE703A983
:101570000120087080E00AE04248006880070028E7
:1015800004D4FFE703A90120087075E0FFE7FFE737
:10159000FFE78649086807229043029A5268104381
:1015A0000860FFF7D3FE0090FFE78048006838210D
:1015B000084002994968C90088420DD0FFE7FFF74B
:1015C000C5FE0099401A3349884204D3FFE703A9B6
:1015D0000320087050E0E8E7FFE701982849096810
:1015E00001221140884221D2FFE7254908680122E3
:1015F0009043019A10430860FFF7A8FE0090FFE7B0
:101600001F48006801210840019988420DD0FFE77A
:10161000FFF79CFE0099401A1E49884204D3FFE759
:1016200003A90320087027E0EAE7FFE702980078A3
:10163000400700280AD5FFE75C4908680722120323
:101640009043029AD26810430860FFE700F03CF82C
:10165000564909680F22120211408A090B4989581C
:101660001F221140C8400E49086009480068FFF772
:1016700091FE03A90870FFE703A8007804B080BDBD
:1016800000200240601002405C100240103100084F
:101690001000002089130000014800687047C04610
:1016A0000400002080B5FFF7F7FF404909680722D2
:1016B000120311408A0A034989581F221140C84069
:1016C00080BDC04650310008B0B58CB0364902A884
:1016D0003CC93CC03CC93CC0344800688006400F4F
:1016E000002817D1FFE7384800680721C9020840E1
:1016F000C10A012088400B902D48006880B2400B41
:1017000001900198810002A840580B99FEF7A3FDB3
:101710000A9046E02548006838210840082803D18F
:10172000FFE728480A903BE020480068382108403D
:10173000202804D1FFE70120C0030A902FE01B48B6
:10174000006838210840182825D1FFE718480068AC
:1017500018490840010C18480068184A104088428F
:1017600004D1FFE70120C0030A9013E0104800688D
:1017700010490840010C12480068104A1040884285
:1017800004D1FFE74B2040020A9002E000200A90BB
:10179000FFE7FFE702E000200A90FFE7FFE7FFE72F
:1017A000FFE70A980CB0B0BD703100080810024085
:1017B000041002400000FF014401FF1FFF01000070
:1017C0004801FF1F00366E010010024080B584B052
:1017D00002900298002804D1FFE703A901200870B5
:1017E0001EE202980078C00700282CD0FFE7FB48D3
:1017F0000068382108400090009808280AD1FFE7C7
:1018000002984068002804D1FFE703A9012008706E
:1018100006E217E0FFE70298406801218904884248
:1018200007D1FFE7EE4908680122920410430860DF
:1018300006E0EB4908680122920490430860FFE744
:10184000FFE7FFE7FFE7029800788007002800D451
:10185000B0E0F54800683821084000900098002862
:1018600057D1FFE7F14800684005002809D5FFE798
:1018700002980069002804D1FFE703A9012008703D
:10188000CEE1EB490868EB4A1040029A9269104396
:101890000860FFF75BFD0190FFE7E4480068400542
:1018A00000280CD4FFE7FFF751FD0199401A0328E7
:1018B00004D3FFE703A903200870B1E1EDE7009826
:1018C000002819D1FFE7D94908680722D2029043BE
:1018D000029A526910430860FFF7F6FED249096880
:1018E0000F22120211408A09D34989581F22114040
:1018F000C840D2490860FFE7D1480068FFF74AFDB9
:10190000002804D0FFE703A90120087088E1FFE761
:101910004FE00298006900282DD0FFE7C34908680E
:101920000722D2029043029A526910430860086865
:101930000122120210430860FFF708FD0190FFE743
:10194000BA480068400500280CD4FFE7FFF7FEFC0A
:101950000199401A032804D3FFE703A90320087064
:101960005EE1EDE7B2490868B24A1040029A926916
:10197000104308601CE0AD49086801221202904340
:101980000860FFF7E3FC0190FFE7A8480068400506
:1019900000280CD5FFE7FFF7D9FC0199401A03286E
:1019A00004D3FFE703A90320087039E1EDE7FFE75F
:1019B000FFE7FFE7029800780007002800D49DE0C9
:1019C000994800683821084018284FD1FFE79D4802
:1019D00000688007002809D5FFE70298C069002841
:1019E00004D1FFE703A90120087019E190490868B4
:1019F000954A1040029A126A120410430860FFF7D9
:101A0000A5FC0190FFE78F480068800700280CD4F0
:101A1000FFE7FFF79BFC0199401A032804D3FFE777
:101A200003A903200870FBE0EDE70098182810D107
:101A3000FFE7FFF749FE7C4909680F2212021140B7
:101A40008A097D4989581F221140C8407B49086096
:101A5000FFE77B480068FFF79DFC002804D0FFE704
:101A600003A901200870DBE0FFE746E00298C069A7
:101A7000002825D0FFE77349086801221043086059
:101A8000FFF764FC0190FFE76E48006880070028BC
:101A90000CD4FFE7FFF75AFC0199401A032804D33E
:101AA000FFE703A903200870BAE0EDE76049086882
:101AB000654A1040029A126A1204104308601BE043
:101AC00060490868012290430860FFF73FFC0190DD
:101AD000FFE75C480068800700280CD5FFE7FFF7A8
:101AE00035FC0199401A032804D3FFE703A903201A
:101AF000087095E0EDE7FFE7FFE7FFE70298007861
:101B00004007002800D487E0474800683821084093
:101B1000202810D1FFE74E4800688007002809D52B
:101B2000FFE702988068002804D1FFE703A901209D
:101B3000087075E06FE00298806800280AD0FFE71F
:101B400042490868032212049043029AD268104363
:101B50000860FFE7FFE702988068012806D1FFE7E9
:101B60003B49086801221043086019E00298806828
:101B700005280AD1FFE736490868042210430860A7
:101B8000086801221043086009E031490868012211
:101B9000904308600868042290430860FFE7FFE76D
:101BA000FFE70298806800281CD0FFE7FFF7CEFB14
:101BB0000190FFE726480068800700280DD4FFE762
:101BC000FFF7C4FB0199401A2249884204D3FFE77A
:101BD00003A90320087023E0ECE71BE00810024093
:101BE00000100240FFF7B2FB0190FFE718480068C1
:101BF000800700280DD5FFE7FFF7A8FB0199401AE1
:101C00001449884204D3FFE703A90320087007E0C2
:101C1000ECE7FFE7FFE7FFE703A900200870FFE715
:101C200003A8007804B080BD0810024000100240F4
:101C3000041002400000FFFF1031000804000020E3
:101C40001000002060100240FFFF00FE1010024054
:101C50005C1002408913000080B582B001900198A9
:101C600001F0F4F802B080BD85B003900291FFE767
:101C70000398407F012804D1FFE704A902200870DF
:101C80003CE0039901204877FFE7FFE70399022032
:101C9000887703980068406801900398006880681E
:101CA0000090019870218843019002980168019882
:101CB00008430190019803990968486003980068F7
:101CC000E24988420ED1FFE70098802188430090C6
:101CD00002984168009808430090009803990968A9
:101CE0008860FFE7039901208877FFE703990020C8
:101CF0004877FFE704A900200870FFE704A80078F0
:101D000005B0704780B582B000900098002804D1DB
:101D1000FFE701A90120087019E00098807F0028E2
:101D200007D1FFE7009900204877009800F014F8E9
:101D3000FFE7009902208877009901C901F0D8F8DF
:101D400000990120887701A900200870FFE701A809
:101D5000007802B080BD000082B001900198006858
:101D6000BA4988420DD1FFE7FFE707480268012121
:101D7000C9020A4302600068084000900098FFE72B
:101D8000FFE702B07047C0464010024082B00190A9
:101D9000019902208877019800688068072108402F
:101DA00000900098062807D0FFE7019801680868AE
:101DB000012210430860FFE7019901208877002085
:101DC00002B0704780B586B004900391FFE7049895
:101DD000407F012804D1FFE705A902200870A7E091
:101DE000049901204877FFE7FFE7049902208877EC
:101DF00004980068806802900298772188430290D6
:101E00000298FF2109028843029002980499096808
:101E10008860039800680190002875D0FFE701985A
:101E2000102871D0FFE7019820286DD0FFE70198B6
:101E3000302869D0FFE70198402858D0FFE7019883
:101E400050283AD0FFE70198602843D0FFE7019877
:101E500070280DD0FFE7019801210903884206D0C0
:101E6000FFE7019801214903884216D053E053E06F
:101E700004980068039B99685A68DB6801F08CF845
:101E800004980068806802900298772108430290C5
:101E900002980499096888603EE004980068039BF2
:101EA00099685A68DB6801F077F8049801688868D7
:101EB00001229203104388602EE004980068039A80
:101EC0005168D26801F098F804980068502101F038
:101ED0007EF821E004980068039A5168D26801F006
:101EE000B3F804980068602101F071F814E00498D8
:101EF0000068039A5168D26801F07EF8049800687F
:101F0000402101F064F807E004980068039909682B
:101F100001F05DF800E0FFE7049901208877FFE712
:101F2000049900204877FFE705A900200870FFE723
:101F300005A8007806B080BDFFE7FEE710B58CB0BD
:101F400000200B900A90099008900790FFE7214825
:101F5000026801210A430260006808400690069862
:101F6000FFE7FFE71B48026802210A43026000689E
:101F7000084005900598FFE7FFE71648026804212E
:101F80000A4302600068084004900498FFE70120BB
:101F900000900790089000200190099003200A907B
:101FA0000D4807A90391FFF76DF8009A0520000777
:101FB000029032242146FFF7B3F9009B019A029860
:101FC00003990794089309920A92FFF75BF80CB003
:101FD00010BDC046341002400004005080B588B0E7
:101FE00000200190079006900590049003900290C5
:101FF000FFF758FB01996748144A0260416081600D
:10200000CA43C26001618161FFF77CFE002802D0F3
:10201000FFE7FFE7FEE70120000304905D4804A905
:10202000FFF7D0FE002802D0FFE7FFE7FEE7002021
:1020300002900390574802A9FFF716FE002802D02D
:10204000FFE7FFE7FEE708B080BDC046002C014077
:102050007047000070B582B0024601A8027000917E
:102060000021405600281BD5FFE701A908780F245E
:10207000204008380322D3431840164A80580025D0
:1020800049578D07EE0EFF25B540A843009DAD01D1
:10209000EDB2B5402843214008391940885015E079
:1020A000002401A908570322D3431840084A805846
:1020B00009578C07E50EFF24AC40A043009CA40107
:1020C000E4B2AC40204319408850FFE702B070BD35
:1020D00000E400E01CED00E089B0089007A8017062
:1020E00006A900200870FFE707AA1078411E1170AA
:1020F000002833D0FFE70898411C0891007805A913
:10210000087004A908200870FFE704A800780028D8
:1021100023D0FFE70699059841400120014003A81C
:10212000017006AA00921178490811700178019196
:102130008C200029029001D1019802900099029A06
:1021400006985040087005A9087840080870FFE715
:102150000498401E04A90870D7E7C5E706A80078D0
:1021600009B0704781B000900A48016800204862B9
:10217000009909480068484308490880FFE7054876
:102180000068406A05490988884201D2FFE7F6E7FE
:1021900001B070473C0300200800002038030020F5
:1021A00083B002900191694600200870FFE76846FD
:1021B000007807280DDCFFE7029869460A78801846
:1021C000C07801998854FFE70098401C6946087060
:1021D000EDE703B0704780B586B005900598012102
:1021E000029100F05BF80299059800F041F87D201B
:1021F0000390C0000190FFF7B5FF059800210491FE
:1022000000F036F80198FFF7ADFF0299059800F04D
:102210002FF803980001FFF7A5FF049805990870AF
:1022200005998870059948700599C87206B080BDF7
:1022300080B584B0039002910398552100F06AFAAA
:1022400001A900200870FFE701A8007807280DDC2D
:10225000FFE70398029901AA1278895C00F05AFA04
:10226000FFE70198401C01A90870EDE704B080BDAC
:1022700082B00190684601700078002805D0FFE721
:10228000019988890969886105E0019988890004B4
:1022900009698861FFE702B07047000084B00390CD
:1022A00002A801702F480068002834D0FFE72D49AC
:1022B000002008600190FFE70198072811DCFFE784
:1022C000039880890199C840012805D1FFE701984A
:1022D000800025490860FFE7FFE70198401C019056
:1022E000EAE708200090FFE700980F2812DCFFE7DC
:1022F000039880890099C840012806D1FFE700981B
:102300008000203818490860FFE7FFE70098401C6C
:102310000090E9E7FFE702A8007800280ED1FFE768
:1023200011480068032282400398016908689043BD
:102330000860039801690868086011E00A480168AC
:1023400003238B4003990A6911689943116000685F
:102350000122824003980169086810430860FFE782
:1023600004B0704700000020D000002081B0009031
:10237000009800690069009989890840411E8841D8
:1023800001B0704780B586B004900498002804D14D
:10239000FFE705A90020087021E003A802900021B2
:1023A000019101700498FFF763FF04980121FFF782
:1023B00075FF0220FFF7D6FE01990498FFF76EFF24
:1023C0000620FFF7CFFE0498FFF7D0FF02990870B0
:1023D0003220FFF7C7FE039805A90870FFE705A89C
:1023E000007806B080BD80B586B0049004980028BF
:1023F00004D1FFE705A9002008701FE003A9002011
:10240000087002A908200870FFE702AA1078411E90
:10241000117000280ED0FFE703A901910878400849
:1024200008700498FFF7AEFF0199C20103981043AA
:102430000870EAE7039805A90870FFE705A8007887
:1024400006B080BD80B584B002900298002804D107
:10245000FFE703A90120087020E002980021009105
:10246000FFF706FF02980121FFF718FF0F20400138
:10247000FFF778FE00990298FFF710FF4620FFF75C
:1024800071FE0298FFF772FF01A90870CD2040008D
:10249000FFF768FE019803A90870FFE703A800781A
:1024A00004B080BD80B58EB00C900BA801700C9864
:1024B000002804D1FFE70DA900200870E4E00AA974
:1024C0000120087009AA0021117008AA117007AA3A
:1024D000117006A908700C988078002800D0BBE025
:1024E0000C98FFF7AFFF00280AD0FFE70C990020F7
:1024F00008700C9988700C9948700DA90870C3E099
:102500000C980BA9097800F005F9FFE70C98FFF784
:1025100039FF05A9029108700C98FFF733FF0146B7
:10252000029804AA11700078012806D1FFE704A8D8
:102530000078012801D1FFE778E005A8007804A918
:102540000978884204D0FFE7059803A9087036E0AF
:102550000AA800780C990978884214DAFFE70C98E9
:1025600008A909784018C17806A800780140012020
:10257000002200920029019001DC0098019001984E
:1025800003A9087009E00AA800780C990978401A94
:102590004142484103A90870FFE703A800780028DA
:1025A0000CD1FFE70A9909A801700078082804DC1B
:1025B000FFE709980C994870FFE7FFE7FFE703A8DA
:1025C0000078012809D1FFE7069A0C9808A9097834
:1025D0004118C8781043C87008E0069A0C9808A9FA
:1025E00009784118C8789043C870FFE70C9803A990
:1025F000097800F04DF80A98401C0AA9087006985E
:10260000410006A801700078002808D1FFE708986B
:10261000401C08A9087006A901200870FFE7FFE721
:10262000FFE708A80078082800DA6FE70AA8007812
:10263000412810DBFFE709980C9908700C98007886
:10264000002804D1FFE70C9901208870FFE707A953
:1026500001200870FFE7FFE707A80078002805D0F1
:10266000FFE70C98C07800280AD1FFE70C990020FA
:1026700008700C9988700C99487007A90870FFE7DA
:1026800007980DA90870FFE70DA800780EB080BD6F
:1026900080B586B0059004A801700598002801D186
:1026A000FFE735E004A80078002818D0FFE7059878
:1026B00000210391FFF7DCFD05980121FFF7EEFDF6
:1026C0000820FFF74FFD03990598FFF7E7FD32203B
:1026D000FFF748FD03990598FFF7E0FD18E005981E
:1026E00000210291FFF7C4FD059801210191FFF738
:1026F000D5FD3920FFF736FD02990598FFF7CEFD8D
:102700000198FFF72FFD02990598FFF7C7FDFFE736
:1027100006B080BD80B584B0039002A80170039814
:10272000002801D1FFE717E001A908200870FFE7A2
:1027300001AA1078411E117000280DD0FFE7039800
:1027400002A90091097801221140FFF7A1FF009929
:10275000087840080870EBE704B080BD80B584B00D
:10276000029001910298002804D1FFE703A90120FB
:1027700008702BE00198002804D1FFE703A901208D
:10278000087023E001994820085A088501991148EA
:10279000086302980199FEF7ABF80146684601709C
:1027A0000078002807D1FFE701996022885CFE23AA
:1027B0001840885406E001996022885C0123184380
:1027C0008854FFE7009803A90870FFE703A8007882
:1027D00004B080BD510D000880B586B0049003910F
:1027E000002000900398002804D1FFE705A90120EC
:1027F00008702FE0039800788007C00F002804D1EC
:10280000FFE705A90120087024E00398007840073D
:10281000C00F00281AD0FFE701A90878FC22104059
:1028200008700398FEF714F9002807D0FFE7039912
:102830006022885C01231843885406E003996022D3
:10284000885CFE2318408854FFE7FFE705A90020B5
:102850000870FFE705A8007806B080BD10B586B007
:10286000049003910398002804D1FFE705A90120F3
:1028700008703AE0049825210A01811880584968B7
:10288000084300282DD0FFE704984B21C900405A87
:10289000002826D0FFE70498972189004058002897
:1028A0001FD0FFE7049A10689721890001915158C1
:1028B00025231C01131912595B6800F09DF9019A38
:1028C00002A90870049B1919002018514860049946
:1028D0004B23DB00C85204998850029805A9087060
:1028E00003E005A900200870FFE705A8007806B0FE
:1028F00010BD0000B0B590B00E900D910E9800285C
:1029000004D1FFE70FA901200870C3E00D9800284B
:1029100004D1FFE70FA901200870BBE00E980D99C4
:1029200008600D994920C2000020885409A9891C1B
:1029300008910790FFE707980E99C97A884200DB53
:10294000A4E00E980799CA006B49891809AAFDF7F7
:1029500017FE01460CA801700078002802D0FFE79E
:1029600000BFFFE7089801780320014000200329F9
:10297000069003DCFFE701200690FFE70698C007FA
:10298000002858D0FFE7089840784007C10F002082
:102990000129059018DCFFE7089840784007C10F2F
:1029A0000020002905900FD4FFE708984178032004
:1029B000014000200329049003DCFFE7012004907C
:1029C000FFE704980590FFE70598C007002832D07C
:1029D000FFE7089840784006810F00200329039004
:1029E00024DCFFE7089840784006810F0020012989
:1029F00003901BDBFFE708984078C006810F00209A
:102A0000022902900FDCFFE708984078C006810F8A
:102A10000120002200920029019001DC0098019021
:102A200001980290FFE702980390FFE70398C00720
:102A3000002826D1FFE707980D9A4921CC00155DA3
:102A400048210B466B43D2183423D0540D98035DB4
:102A50000A465A438218114890630E980D9B1A5DDE
:102A600051435918521C1A550831FDF741FF0146D0
:102A70000CA801700078002802D0FFE700BFFFE734
:102A8000FFE7FFE70798401C079054E70FA90020D5
:102A90000870FFE70FA8007810B0B0BDD10B000898
:102AA00080B586B000200390059011480290012166
:102AB000818110490161104A0192A0231F21D15444
:102AC000FFF789FB01980299FDF79EFD02980B49DB
:102AD0002922120200F014F80298A0490491FFF78D
:102AE00009FF03990498FFF7B9FE06B080BDC04600
:102AF000BC000020000400501800002060030020EB
:102B000010B588B00690059104A8028006980028A8
:102B100004D1FFE707A90120087068E005980028A4
:102B200004D1FFE707A90120087060E0049803A919
:102B30000880069805990860059A03993520C00019
:102B4000019011500599085A502288520599885CC5
:102B5000FC242040885405990120029008660698BC
:102B600005990831FFF7FAFD01990298059A515A23
:102B7000B823D152059AD15C2140491CD154059902
:102B8000C8228850069805997031FFF7E7FD019932
:102B90000298059A515A09235B01D152059AD15CDA
:102BA0002140891CD154059913221201885006989E
:102BB0000599D831FFF7D2FD01990298059A515A2B
:102BC0003123DB00D152059AD15C03242143D15437
:102BD00005993322D2008850069805990522920162
:102BE0008918FFF7BBFD07A900200870FFE707A8B9
:102BF000007808B010BD000010B59AB01890179179
:102C0000159314921898002804D1FFE719A9012000
:102C100008705AE01798002804D1FFE719A901208D
:102C2000087052E01498159A17994A620862179929
:102C30004820085A08851799264808631898179954
:102C4000FDF756FE014601A80170007800280AD061
:102C5000FFE717996022885C012318438854019884
:102C600019A9087031E017984821425A03231146E8
:102C7000FEF77CF9014601A801700078002804D015
:102C8000FFE7019819A908701FE017991248086317
:102C900018981799FDF72CFE014601A801700078DD
:102CA000002807D1FFE717996022885CFE231840AF
:102CB000885406E017996022885C012318438854E1
:102CC000FFE7019819A90870FFE719A800781AB062
:102CD00010BDC046210C0008510D000880B586B01B
:102CE00004900498002804D1FFE705A9012008708A
:102CF0002FE004980068012100220292FEF7D6F826
:102D000003A90191087004990868083100F028F8B7
:102D10000199087004990868703100F021F8019950
:102D2000087004990868D83100F01AF80199087001
:102D30000499086805229201891800F011F8019A97
:102D4000029910700548FFF789FD039805A90870DE
:102D5000FFE705A8007806B080BDC046D800002077
:102D600080B584B0029001910198002804D1FFE75A
:102D700003A9012008703AE00198416D006D0843F5
:102D800000280DD0FFE7029801994B6D0A6DFFF7FF
:102D900033FF694608700199002048650865FFE720
:102DA0000198806D002810D0FFE70198FDF70CFE18
:102DB0000146684601700078002805D0FFE70298B8
:102DC0000199FFF709FDFFE7FFE70198C06D0028B3
:102DD00009D0FFE701990020C865019800F00BF8C1
:102DE00069460870FFE7009803A90870FFE703A889
:102DF000007804B080BD80B584B0029002980028AD
:102E000004D1FFE703A90120087019E0029800220D
:102E100003231146FEF7AAF8014601A801700078C5
:102E2000002804D0FFE7019803A9087008E0029881
:102E3000FDF74AFE01A90870019803A90870FFE791
:102E400003A8007804B080BD7047704780B584B097
:102E500002900298401E000E002803D0FFE70120D8
:102E6000039011E00298401E09490860002001907B
:102E7000C0430321FFF7EEF8019806490860064AAF
:102E8000072111600390FFE7039804B080BDC0469E
:102E900014E000E018E000E010E000E080B5FEF78C
:102EA00059FA80BD80B50C4908680C4A10400C4A9C
:102EB00012681043086008680A4A10400A4A1268FB
:102EC0001204104308600120C0060849086064200D
:102ED000FEF7A4F880BDC046041002400000FFFFCA
:102EE0000001FF1FFFFF00FE4401FF1F08ED00E08F
:102EF00083B00290019102980068009002982449E2
:102F000088420AD1FFE70098702188430090019819
:102F10004168009808430090FFE702981C498842E6
:102F200005D0FFE702981B4988420BD1FFE70098C4
:102F300003210902884300900198C1680098084362
:102F40000090FFE700988021884301994969084370
:102F50000090009802990860019880680299C86200
:102F6000019800680299886202980949884205D050
:102F7000FFE702980749884205D1FFE701980069F9
:102F800002990863FFE702990120486103B0704786
:102F9000002C01400020004085B004900391029273
:102FA00001930498806800900098FF2109028843EB
:102FB000009003990298019A12021043014300986D
:102FC0000843009000980499886005B0704783B06A
:102FD00002900191029880680090009870218843C7
:102FE0000090019800990843072108430090009839
:102FF0000299886003B0704785B0049003910292F3
:103000000498006A00900499086A012290430862BB
:103010000498806901900198F021884301900298FA
:10302000010101980843019000980A21884300900B
:1030300003990098084300900198049988610098CA
:103040000499086205B0704785B00490039102921C
:103050000499086A102290430862049880690190DC
:103060000498006A009001980F2109038843019099
:10307000029801030198084301900098A021884319
:10308000009003980101009808430090019804996A
:10309000886100980499086205B0704780B582B0D5
:1030A000002001900E4908680122D20210430860F6
:1030B000FEF75AF9FDF744F9FEF740FFFEF78EFFE1
:1030C0000848FEF763FEFFF7EBFCFFE706490868D8
:1030D0000222504008600548FFF700FEF6E7C046B0
:1030E0000C5801403C0300201400005060030020F5
:1030F00002E008C8121F08C1002AFAD170477047C1
:10310000002001E001C1121F002AFBD1704700001E
:1031100000000000000000000000000000000000AF
:10312000000000000000000000000000000000009F
:103130000100000002000000030000000400000085
:103140000600000007000000080000000900000061
:10315000000000000000000000000000000000006F
:103160000100000002000000030000000400000055
:10317000000000000000000000000000000000004F
:1031800000366E010000000000000000000000009A
:10319000B03100080000002018000000F0300008E6
:1031A000C83100081800002008090000003100089C
:1031B0000100000000366E01180000000100000050
:0831C000040000000000000003
:04000005080000C12E
:00000001FF
